******************************************************************************
                  TI ARM Linker PC v20.2.4                     
******************************************************************************
>> Linked Fri Mar 19 14:52:22 2021

OUTPUT FILE NAME:   <enet_udpecho_client_lwip.out>
ENTRY POINT SYMBOL: "_c_int00_noargs"  address: 0000a0b1


MEMORY CONFIGURATION

         name            origin    length      used     unused   attr    fill
----------------------  --------  ---------  --------  --------  ----  --------
  FLASH                 00000000   00100000  0000ad7a  000f5286  R  X
  SRAM                  20000000   00040000  0001830f  00027cf1  RW X


SEGMENT ALLOCATION MAP

run origin  load origin   length   init length attrs members
----------  ----------- ---------- ----------- ----- -------
00000000    00000000    0000ad80   0000ad80    r-x
  00000000    00000000    00000200   00000200    r-- .intvecs
  00000200    00000200    0000a776   0000a776    r-x .text
  0000a978    0000a978    000003ac   000003ac    r-- .const
  0000ad28    0000ad28    00000058   00000058    r-- .cinit
20000000    20000000    00018310   00000000    rw-
  20000000    20000000    00017a9f   00000000    rw- .bss
  20017aa0    20017aa0    00000800   00000000    rw- .stack
  200182a0    200182a0    00000070   00000000    rw- .data


SECTION ALLOCATION MAP

 output                                  attributes/
section   page    origin      length       input sections
--------  ----  ----------  ----------   ----------------
.intvecs   0    00000000    00000200     
                  00000000    00000200     startup_ccs.obj (.intvecs)

.text      0    00000200    0000a776     
                  00000200    00000bc4     lwiplib.obj (.text:tcp_receive)
                  00000dc4    0000060c     lwiplib.obj (.text:tcp_process)
                  000013d0    00000580     lwiplib.obj (.text:tcp_input)
                  00001950    00000448     lwiplib.obj (.text:tcp_slowtmr)
                  00001d98    00000438     ustdlib.obj (.text:uvsnprintf)
                  000021d0    000003f0     lwiplib.obj (.text:dhcp_parse_reply)
                  000025c0    0000030c     uartstdio.obj (.text:UARTvprintf)
                  000028cc    00000298     lwiplib.obj (.text:udp_input)
                  00002b64    00000290     lwiplib.obj (.text:ip_input)
                  00002df4    00000288     lwiplib.obj (.text:tivaif_receive)
                  0000307c    0000026c     pinout.obj (.text:PinoutSet)
                  000032e8    00000244     lwiplib.obj (.text:tcp_output)
                  0000352c    0000023c     lwiplib.obj (.text:tcp_close_shutdown)
                  00003768    00000228     lwiplib.obj (.text:etharp_find_entry)
                  00003990    0000020e     lwiplib.obj (.text:pbuf_alloc)
                  00003b9e    00000206     lwiplib.obj (.text:ipaddr_aton)
                  00003da4    00000200     driverlib.lib : sysctl.obj (.text:SysCtlClockFreqSet)
                  00003fa4    000001fc     lwiplib.obj (.text:dhcp_create_msg)
                  000041a0    000001e4     lwiplib.obj (.text:icmp_input)
                  00004384    000001dc     enet_udpecho_client_lwip.obj (.text:main)
                  00004560    000001c4     lwiplib.obj (.text:etharp_query)
                  00004724    000001c0     lwiplib.obj (.text:etharp_arp_input)
                  000048e4    000001b8     lwiplib.obj (.text:tivaif_transmit)
                  00004a9c    000001b0     lwiplib.obj (.text:InitDMADescriptors)
                  00004c4c    000001a8     lwiplib.obj (.text:etharp_output)
                  00004df4    0000019c     lwiplib.obj (.text:mem_trim)
                  00004f90    00000188     lwiplib.obj (.text:mem_malloc)
                  00005118    00000178     lwiplib.obj (.text:tcp_enqueue_flags)
                  00005290    00000170     lwiplib.obj (.text:tcp_listen_input)
                  00005400    0000016c     driverlib.lib : gpio.obj (.text:GPIOPadConfigSet)
                  0000556c    0000015c     enet_udpecho_client_lwip.obj (.text:UdpClientInit)
                  000056c8    0000015c     lwiplib.obj (.text:autoip_tmr)
                  00005824    0000014e     lwiplib.obj (.text:dhcp_bind)
                  00005972    00000002     startup_ccs.obj (.text:FaultISR)
                  00005974    00000138     lwiplib.obj (.text:dhcp_recv)
                  00005aac    0000012c     lwiplib.obj (.text:tcp_output_segment)
                  00005bd8    00000128     lwiplib.obj (.text:tcp_alloc)
                  00005d00    0000011c     lwiplib.obj (.text:pbuf_copy)
                  00005e1c    00000118     lwiplib.obj (.text:udp_sendto_if)
                  00005f34    00000114     lwiplib.obj (.text:dhcp_select)
                  00006048    00000108     lwiplib.obj (.text:dhcp_discover)
                  00006150    00000104     lwiplib.obj (.text:etharp_raw)
                  00006254    00000104     lwiplib.obj (.text:memp_init)
                  00006358    00000104     lwiplib.obj (.text:tcp_parseopt)
                  0000645c    000000fc     lwiplib.obj (.text:dhcp_start)
                  00006558    000000fc     lwiplib.obj (.text:etharp_update_arp_entry)
                  00006654    000000f8     lwiplib.obj (.text:ethernet_input)
                  0000674c    000000f0     lwiplib.obj (.text:lwIPInit)
                  0000683c    000000ec     lwiplib.obj (.text:ip_output_if)
                  00006928    000000e8     lwiplib.obj (.text:dhcp_release)
                  00006a10    000000e8     lwiplib.obj (.text:pbuf_copy_partial)
                  00006af8    000000e8     lwiplib.obj (.text:tcp_create_segment)
                  00006be0    000000e4     lwiplib.obj (.text:lwIPServiceTimers)
                  00006cc4    000000dc     lwiplib.obj (.text:pbuf_header)
                  00006da0    000000dc     lwiplib.obj (.text:tivaif_hwinit)
                  00006e7c    000000d8     lwiplib.obj (.text:tcp_zero_window_probe)
                  00006f54    000000d4     lwiplib.obj (.text:sys_timeout)
                  00007028    000000d0     lwiplib.obj (.text:dhcp_reboot)
                  000070f8    000000c0     lwiplib.obj (.text:etharp_tmr)
                  000071b8    000000c0     lwiplib.obj (.text:netif_set_ipaddr)
                  00007278    000000c0     lwiplib.obj (.text:udp_bind)
                  00007338    000000be     lwiplib.obj (.text:dhcp_timeout)
                  000073f6    00000002     startup_ccs.obj (.text:IntDefaultHandler)
                  000073f8    000000bc     lwiplib.obj (.text:dhcp_handle_ack)
                  000074b4    000000bc     lwiplib.obj (.text:tcp_abandon)
                  00007570    000000bc     lwiplib.obj (.text:tcp_process_refused_data)
                  0000762c    000000b6     lwiplib.obj (.text:pbuf_realloc)
                  000076e2    00000002     startup_ccs.obj (.text:NmiSR)
                  000076e4    000000b4     lwiplib.obj (.text:dhcp_rebind)
                  00007798    000000b4     lwiplib.obj (.text:raw_input)
                  0000784c    000000b4     lwiplib.obj (.text:tcp_oos_insert_segment)
                  00007900    000000b2     lwiplib.obj (.text:dhcp_renew)
                  000079b2    000000b2     lwiplib.obj (.text:lwip_standard_chksum)
                  00007a64    000000b0     lwiplib.obj (.text:pbuf_take)
                  00007b14    000000b0     lwiplib.obj (.text:tcp_timewait_input)
                  00007bc4    000000ac     lwiplib.obj (.text:autoip_arp_reply)
                  00007c70    000000ac     lwiplib.obj (.text:dhcp_decline)
                  00007d1c    000000ac     lwiplib.obj (.text:plug_holes)
                  00007dc8    000000ac     lwiplib.obj (.text:tcp_output_alloc_header)
                  00007e74    000000a8     lwiplib.obj (.text:lwIPLinkDetect)
                  00007f1c    000000a8     lwiplib.obj (.text:memp_malloc)
                  00007fc4    000000a8     lwiplib.obj (.text:pbuf_free)
                  0000806c    000000a8     lwiplib.obj (.text:tivaif_process_transmit)
                  00008114    000000a0     lwiplib.obj (.text:icmp_send_response)
                  000081b4    000000a0     lwiplib.obj (.text:inet_chksum_pbuf)
                  00008254    000000a0     lwiplib.obj (.text:tcp_pcb_remove)
                  000082f4    000000a0     lwiplib.obj (.text:tivaif_process_phy_interrupt)
                  00008394    0000009c     rtsv7M4_T_le_v4SPD16_eabi.lib : memcpy_t2.asm.obj (.text)
                  00008430    00000098     lwiplib.obj (.text:tcp_rst)
                  000084c8    00000094     lwiplib.obj (.text:autoip_start)
                  0000855c    00000094     enet_udpecho_client_lwip.obj (.text:lwIPHostTimerHandler)
                  000085f0    0000008e     lwiplib.obj (.text:tcp_rexmit_fast)
                  0000867e    00000002     lwiplib.obj (.text:netif_init)
                  00008680    0000008c     lwiplib.obj (.text:lwIPEthernetIntHandler)
                  0000870c    0000008c     lwiplib.obj (.text:udp_connect)
                  00008798    00000088     lwiplib.obj (.text:mem_free)
                  00008820    00000088     lwiplib.obj (.text:tcp_fasttmr)
                  000088a8    00000084     lwiplib.obj (.text:ip_route)
                  0000892c    00000084     lwiplib.obj (.text:lwIPPrivateInit)
                  000089b0    00000084     lwiplib.obj (.text:netif_add)
                  00008a34    00000084     lwiplib.obj (.text:tcp_kill_prio)
                  00008ab8    00000080     lwiplib.obj (.text:etharp_output_to_arp_index)
                  00008b38    0000007c     lwiplib.obj (.text:autoip_start_probing)
                  00008bb4    0000007c     lwiplib.obj (.text:mem_init)
                  00008c30    0000007c     lwiplib.obj (.text:tcp_rexmit)
                  00008cac    0000007a     rtsv7M4_T_le_v4SPD16_eabi.lib : memset_t2.asm.obj (.text)
                  00008d26    00000002                                   : div0.asm.obj (.text)
                  00008d28    00000078     driverlib.lib : emac.obj (.text:EMACInit)
                  00008da0    00000076     lwiplib.obj (.text:tcp_update_rcv_ann_wnd)
                  00008e16    00000002     lwiplib.obj (.text:stats_init)
                  00008e18    00000074     uartstdio.obj (.text:UARTStdioConfig)
                  00008e8c    00000074     lwiplib.obj (.text:autoip_create_addr)
                  00008f00    00000072     lwiplib.obj (.text:dhcp_option_long)
                  00008f72    0000006c     lwiplib.obj (.text:ip4_addr_isbroadcast)
                  00008fde    00000002     lwiplib.obj (.text:tcp_init)
                  00008fe0    0000006c     lwiplib.obj (.text:udp_new_port)
                  0000904c    0000006a     lwiplib.obj (.text:tcp_pcb_purge)
                  000090b6    00000002     lwiplib.obj (.text:udp_init)
                  000090b8    00000068     driverlib.lib : interrupt.obj (.text:IntEnable)
                  00009120    00000068     rtsv7M4_T_le_v4SPD16_eabi.lib : copy_decompress_lzss.c.obj (.text:decompress:lzss:__TI_decompress_lzss)
                  00009188    00000068     lwiplib.obj (.text:tivaif_check_pbuf)
                  000091f0    00000066     lwiplib.obj (.text:tcp_send_empty_ack)
                  00009256    00000002     --HOLE-- [fill = 0]
                  00009258    00000064     uartstdio.obj (.text:UARTwrite)
                  000092bc    00000064     lwiplib.obj (.text:etharp_cleanup_netif)
                  00009320    00000062     lwiplib.obj (.text:dhcp_network_changed)
                  00009382    0000005c     lwiplib.obj (.text:tcp_send_fin)
                  000093de    00000002     --HOLE-- [fill = 0]
                  000093e0    00000058     driverlib.lib : emac.obj (.text:EMACPHYConfigSet)
                  00009438    00000058     lwiplib.obj (.text:tcp_keepalive)
                  00009490    00000058     lwiplib.obj (.text:tivaif_interrupt)
                  000094e8    00000058     lwiplib.obj (.text:udp_remove)
                  00009540    00000058     ustdlib.obj (.text:ustrncpy)
                  00009598    00000054     lwiplib.obj (.text:dhcp_fine_tmr)
                  000095ec    00000054     lwiplib.obj (.text:memp_free)
                  00009640    00000054     lwiplib.obj (.text:netif_set_link_up)
                  00009694    00000054     lwiplib.obj (.text:tcp_kill_timewait)
                  000096e8    00000052     lwiplib.obj (.text:dhcp_option_trailer)
                  0000973a    00000052     lwiplib.obj (.text:dhcp_stop)
                  0000978c    00000050     driverlib.lib : sysctl.obj (.text:SysCtlPeripheralReset)
                  000097dc    00000050     lwiplib.obj (.text:dhcp_coarse_tmr)
                  0000982c    00000050     lwiplib.obj (.text:sys_timeouts_init)
                  0000987c    00000050     lwiplib.obj (.text:tcp_rexmit_rto)
                  000098cc    0000004c     enet_udpecho_client_lwip.obj (.text:DisplayIPAddress)
                  00009918    0000004c     lwiplib.obj (.text:ip_output)
                  00009964    00000048     driverlib.lib : sysctl.obj (.text:_SysCtlFrequencyGet)
                  000099ac    00000048     lwiplib.obj (.text:dhcp_check)
                  000099f4    00000048     lwiplib.obj (.text:etharp_free_entry)
                  00009a3c    00000048     lwiplib.obj (.text:tcp_recved)
                  00009a84    00000046     lwiplib.obj (.text:pbuf_cat)
                  00009aca    00000002     --HOLE-- [fill = 0]
                  00009acc    00000044     rtsv7M4_T_le_v4SPD16_eabi.lib : autoinit.c.obj (.text:__TI_auto_init_nobinit_nopinit:__TI_auto_init_nobinit_nopinit)
                  00009b10    00000044     lwiplib.obj (.text:dhcp_option_short)
                  00009b54    00000044     lwiplib.obj (.text:etharp_send_ip)
                  00009b98    00000044     lwiplib.obj (.text:tcp_eff_send_mss)
                  00009bdc    00000044     lwiplib.obj (.text:tivaif_init)
                  00009c20    00000044     lwiplib.obj (.text:udp_sendto)
                  00009c64    00000040     rtsv7M4_T_le_v4SPD16_eabi.lib : u_divt2.asm.obj (.text)
                  00009ca4    0000003e     lwiplib.obj (.text:dhcp_option)
                  00009ce2    00000002     --HOLE-- [fill = 0]
                  00009ce4    0000003c     enet_udpecho_client_lwip.obj (.text:UdpEchoRecv)
                  00009d20    0000003c     lwiplib.obj (.text:autoip_arp_probe)
                  00009d5c    0000003c     lwiplib.obj (.text:autoip_bind)
                  00009d98    0000003c     lwiplib.obj (.text:dhcp_handle_nak)
                  00009dd4    0000003c     lwiplib.obj (.text:netif_set_up)
                  00009e10    0000003a     driverlib.lib : emac.obj (.text:EMACIntEnable)
                  00009e4a    0000003a     lwiplib.obj (.text:autoip_handle_arp_conflict)
                  00009e84    0000003a     lwiplib.obj (.text:tcp_recv_null)
                  00009ebe    00000002     --HOLE-- [fill = 0]
                  00009ec0    00000038     driverlib.lib : emac.obj (.text:EMACConfigSet)
                  00009ef8    00000038                   : sysctl.obj (.text:SysCtlPeripheralReady)
                  00009f30    00000038     lwiplib.obj (.text:autoip_arp_announce)
                  00009f68    00000038     lwiplib.obj (.text:dhcp_handle_offer)
                  00009fa0    00000038     lwiplib.obj (.text:etharp_request)
                  00009fd8    00000038     lwiplib.obj (.text:tcp_timer_needed)
                  0000a010    00000038     lwiplib.obj (.text:tcpip_tcp_timer)
                  0000a048    00000034     driverlib.lib : emac.obj (.text:EMACConfigGet)
                  0000a07c    00000034                   : emac.obj (.text:EMACIntClear)
                  0000a0b0    00000034     rtsv7M4_T_le_v4SPD16_eabi.lib : boot_cortex_m.c.obj (.text:_c_int00_noargs:_c_int00_noargs)
                  0000a0e4    00000032     ustdlib.obj (.text:usprintf)
                  0000a116    00000030     lwiplib.obj (.text:dhcp_arp_reply)
                  0000a146    0000002e     lwiplib.obj (.text:dhcp_set_state)
                  0000a174    0000002e     lwiplib.obj (.text:netif_set_down)
                  0000a1a2    0000002e     lwiplib.obj (.text:pbuf_clen)
                  0000a1d0    0000002c     driverlib.lib : emac.obj (.text:EMACIntStatus)
                  0000a1fc    0000002c                   : gpio.obj (.text:GPIODirModeSet)
                  0000a228    0000002c     lwiplib.obj (.text:lwip_htonl)
                  0000a254    0000002a     lwiplib.obj (.text:dhcp_t1_timeout)
                  0000a27e    0000002a     lwiplib.obj (.text:dhcp_t2_timeout)
                  0000a2a8    0000002a     lwiplib.obj (.text:netif_set_addr)
                  0000a2d2    0000002a     lwiplib.obj (.text:tcp_seg_copy)
                  0000a2fc    00000028     lwiplib.obj (.text:lwIPTimer)
                  0000a324    00000026     driverlib.lib : emac.obj (.text:EMACPHYRead)
                  0000a34a    00000026                   : emac.obj (.text:EMACPHYWrite)
                  0000a370    00000024                   : interrupt.obj (.text:IntPrioritySet)
                  0000a394    00000024     uartstdio.obj (.text:UARTprintf)
                  0000a3b8    00000024     lwiplib.obj (.text:dhcp_delete_msg)
                  0000a3dc    00000024     lwiplib.obj (.text:dhcp_option_byte)
                  0000a400    00000024     lwiplib.obj (.text:lwip_htons)
                  0000a424    00000024     rtsv7M4_T_le_v4SPD16_eabi.lib : memcmp.c.obj (.text:memcmp)
                  0000a448    00000022     lwiplib.obj (.text:netif_set_link_down)
                  0000a46a    00000022     lwiplib.obj (.text:pbuf_ref)
                  0000a48c    00000022     lwiplib.obj (.text:udp_new)
                  0000a4ae    00000002     --HOLE-- [fill = 0]
                  0000a4b0    00000020     driverlib.lib : sysctl.obj (.text:_SysCtlMemTimingGet)
                  0000a4d0    00000020     lwiplib.obj (.text:autoip_network_changed)
                  0000a4f0    00000020     lwiplib.obj (.text:lwip_init)
                  0000a510    00000020     lwiplib.obj (.text:pbuf_pool_is_empty)
                  0000a530    00000020     lwiplib.obj (.text:tcp_close)
                  0000a550    00000020     lwiplib.obj (.text:tcp_seg_free)
                  0000a570    00000020     lwiplib.obj (.text:tcp_segs_free)
                  0000a590    00000020     lwiplib.obj (.text:tcp_tmr)
                  0000a5b0    00000020     lwiplib.obj (.text:udp_disconnect)
                  0000a5d0    0000001e     driverlib.lib : emac.obj (.text:EMACAddrGet)
                  0000a5ee    00000002     --HOLE-- [fill = 0]
                  0000a5f0    0000001c     lwiplib.obj (.text:arp_timer)
                  0000a60c    0000001c     lwiplib.obj (.text:dhcp_timer_coarse)
                  0000a628    0000001c     lwiplib.obj (.text:dhcp_timer_fine)
                  0000a644    0000001c     lwiplib.obj (.text:lwIPLocalIPAddrGet)
                  0000a660    0000001c     lwiplib.obj (.text:netif_set_gw)
                  0000a67c    0000001c     lwiplib.obj (.text:netif_set_netmask)
                  0000a698    0000001c     lwiplib.obj (.text:sys_arch_unprotect)
                  0000a6b4    0000001c     lwiplib.obj (.text:tcp_next_iss)
                  0000a6d0    0000001a     driverlib.lib : gpio.obj (.text:GPIOPinTypeGPIOOutput)
                  0000a6ea    0000001a     lwiplib.obj (.text:udp_recv)
                  0000a704    00000018     lwiplib.obj (.text:autoip_timer)
                  0000a71c    00000018     lwiplib.obj (.text:inet_chksum)
                  0000a734    00000018     lwiplib.obj (.text:ipaddr_addr)
                  0000a74c    00000018     lwiplib.obj (.text:udp_send)
                  0000a764    00000016     driverlib.lib : emac.obj (.text:EMACReset)
                  0000a77a    00000016                   : emac.obj (.text:EMACRxEnable)
                  0000a790    00000016                   : emac.obj (.text:EMACTxEnable)
                  0000a7a6    00000016                   : gpio.obj (.text:GPIOPinTypeEthernetLED)
                  0000a7bc    00000016     lwiplib.obj (.text:autoip_restart)
                  0000a7d2    00000016     lwiplib.obj (.text:autoip_stop)
                  0000a7e8    00000016     lwiplib.obj (.text:icmp_dest_unreach)
                  0000a7fe    00000016     lwiplib.obj (.text:pbuf_chain)
                  0000a814    00000014     driverlib.lib : flash.obj (.text:FlashUserGet)
                  0000a828    00000014                   : systick.obj (.text:SysTickEnable)
                  0000a83c    00000014                   : systick.obj (.text:SysTickIntEnable)
                  0000a850    00000014     enet_udpecho_client_lwip.obj (.text:SysTickIntHandler)
                  0000a864    00000014     lwiplib.obj (.text:netif_set_default)
                  0000a878    00000014     rtsv7M4_T_le_v4SPD16_eabi.lib : strlen.c.obj (.text:strlen)
                  0000a88c    00000010     driverlib.lib : emac.obj (.text:EMACFrameFilterSet)
                  0000a89c    00000010                   : interrupt.obj (.text:IntMasterEnable)
                  0000a8ac    00000010                   : systick.obj (.text:SysTickPeriodSet)
                  0000a8bc    00000010     lwiplib.obj (.text:lwip_ntohs)
                  0000a8cc    00000010     lwiplib.obj (.text:sys_arch_protect)
                  0000a8dc    0000000e     rtsv7M4_T_le_v4SPD16_eabi.lib : copy_decompress_none.c.obj (.text:decompress:none:__TI_decompress_none)
                  0000a8ea    0000000e     lwiplib.obj (.text:tcp_abort)
                  0000a8f8    0000000c     driverlib.lib : cpu.obj (.text:CPUcpsie)
                  0000a904    0000000c                   : sysctl.obj (.text:SysCtlMOSCConfigSet)
                  0000a910    0000000c     rtsv7M4_T_le_v4SPD16_eabi.lib : copy_zero_init.c.obj (.text:decompress:ZI:__TI_zero_init)
                  0000a91c    0000000c     lwiplib.obj (.text:lwip_ntohl)
                  0000a928    0000000c     lwiplib.obj (.text:sys_now)
                  0000a934    00000008     driverlib.lib : emac.obj (.text:EMACPowerManagementStatusGet)
                  0000a93c    00000008                   : emac.obj (.text:EMACTxDMAPollDemand)
                  0000a944    00000006                   : emac.obj (.text:EMACRxDMADescriptorListSet)
                  0000a94a    00000006                   : emac.obj (.text:EMACTimestampIntStatus)
                  0000a950    00000006                   : emac.obj (.text:EMACTxDMADescriptorListSet)
                  0000a956    00000006                   : gpio.obj (.text:GPIOPinRead)
                  0000a95c    00000006                   : gpio.obj (.text:GPIOPinWrite)
                  0000a962    00000006     startup_ccs.obj (.text:ResetISR)
                  0000a968    00000006     driverlib.lib : sysctl.obj (.text:SysCtlDelay)
                  0000a96e    00000004     rtsv7M4_T_le_v4SPD16_eabi.lib : pre_init.c.obj (.text:_system_pre_init)
                  0000a972    00000004                                   : exit.c.obj (.text:abort:abort)

.const     0    0000a978    000003ac     
                  0000a978    000001b0     driverlib.lib : sysctl.obj (.const:g_pppui32XTALtoVCO)
                  0000ab28    0000009c                   : interrupt.obj (.const:g_pui32Regs)
                  0000abc4    0000006c                   : sysctl.obj (.const:g_pui32Xtals)
                  0000ac30    00000030                   : sysctl.obj (.const:g_sXTALtoMEMTIM)
                  0000ac60    00000018                   : emac.obj (.const:g_pi16MIIClockDiv)
                  0000ac78    00000014                   : interrupt.obj (.const:g_pui32EnRegs)
                  0000ac8c    00000012     uartstdio.obj (.const:.string)
                  0000ac9e    00000002     --HOLE-- [fill = 0]
                  0000aca0    00000012     ustdlib.obj (.const:.string)
                  0000acb2    00000010     lwiplib.obj (.const:memp_num)
                  0000acc2    00000010     lwiplib.obj (.const:memp_sizes)
                  0000acd2    0000000d     lwiplib.obj (.const:.string:tcp_backoff)
                  0000acdf    00000001     --HOLE-- [fill = 0]
                  0000ace0    0000000c     uartstdio.obj (.const:g_ui32UARTBase)
                  0000acec    0000000c     uartstdio.obj (.const:g_ui32UARTPeriph)
                  0000acf8    00000008     driverlib.lib : sysctl.obj (.const:g_pui32VCOFrequencies)
                  0000ad00    00000007     lwiplib.obj (.const:.string:tcp_persist_backoff)
                  0000ad07    00000006     lwiplib.obj (.const:ethbroadcast)
                  0000ad0d    00000006     lwiplib.obj (.const:ethzero)
                  0000ad13    00000001     --HOLE-- [fill = 0]
                  0000ad14    00000004     lwiplib.obj (.const:ip_addr_any)
                  0000ad18    00000004     lwiplib.obj (.const:ip_addr_broadcast)
                  0000ad1c    00000004     uartstdio.obj (.const)
                  0000ad20    00000004     ustdlib.obj (.const)

.cinit     0    0000ad28    00000058     
                  0000ad28    0000002f     (.cinit..data.load) [load image, compression = lzss]
                  0000ad57    00000001     --HOLE-- [fill = 0]
                  0000ad58    0000000c     (__TI_handler_table)
                  0000ad64    00000004     --HOLE-- [fill = 0]
                  0000ad68    00000008     (.cinit..bss.load) [load image, compression = zero_init]
                  0000ad70    00000010     (__TI_cinit_table)

.init_array 
*          0    00000000    00000000     UNINITIALIZED

.bss       0    20000000    00017a9f     UNINITIALIZED
                  20000000    0001001c     (.common:ram_heap)
                  2001001c    000072d4     lwiplib.obj (.bss:memp_memory)
                  200172f0    00000360     (.common:g_pTxDescriptors)
                  20017650    00000120     (.common:g_pRxDescriptors)
                  20017770    00000120     (.common:lwip_stats)
                  20017890    000000c8     lwiplib.obj (.bss:arp_table)
                  20017958    00000050     lwiplib.obj (.bss)
                  200179a8    00000038     lwiplib.obj (.bss:g_sNetIF)
                  200179e0    00000028     (.common:dhcp_rx_options_val)
                  20017a08    00000020     lwiplib.obj (.bss:memp_tab)
                  20017a28    00000010     lwiplib.obj (.bss:inseg)
                  20017a38    0000000c     (.common:dhcp_rx_options_given)
                  20017a44    00000008     (.common:g_scbFlag)
                  20017a4c    00000004     (.common:current_header)
                  20017a50    00000004     (.common:current_iphdr_dest)
                  20017a54    00000004     (.common:current_iphdr_src)
                  20017a58    00000004     (.common:current_netif)
                  20017a5c    00000004     (.common:g_pfnTimerHandler)
                  20017a60    00000004     (.common:g_ui32AbnormalInts)
                  20017a64    00000004     (.common:g_ui32IPAddress)
                  20017a68    00000004     (.common:g_ui32NormalInts)
                  20017a6c    00000004     (.common:g_ui32SysClock)
                  20017a70    00000004     (.common:netif_default)
                  20017a74    00000004     (.common:netif_list)
                  20017a78    00000004     (.common:tcp_active_pcbs)
                  20017a7c    00000004     (.common:tcp_bound_pcbs)
                  20017a80    00000004     (.common:tcp_input_pcb)
                  20017a84    00000004     (.common:tcp_listen_pcbs)
                  20017a88    00000004     (.common:tcp_ticks)
                  20017a8c    00000004     (.common:tcp_tmp_pcb)
                  20017a90    00000004     (.common:tcp_tw_pcbs)
                  20017a94    00000004     (.common:udp_pcbs)
                  20017a98    00000004     (.common:upcb)
                  20017a9c    00000001     (.common:g_bLED)
                  20017a9d    00000001     (.common:pbuf_free_ooseq_pending)
                  20017a9e    00000001     (.common:tcp_active_pcbs_changed)

.data      0    200182a0    00000070     UNINITIALIZED
                  200182a0    00000038     lwiplib.obj (.data)
                  200182d8    00000010     lwiplib.obj (.data:g_RxDescList)
                  200182e8    00000010     lwiplib.obj (.data:g_TxDescList)
                  200182f8    0000000c     lwiplib.obj (.data:g_StellarisIFData)
                  20018304    00000005     uartstdio.obj (.data)
                  20018309    00000003     --HOLE--
                  2001830c    00000004     enet_udpecho_client_lwip.obj (.data)

.stack     0    20017aa0    00000800     UNINITIALIZED
                  20017aa0    00000004     rtsv7M4_T_le_v4SPD16_eabi.lib : boot_cortex_m.c.obj (.stack)
                  20017aa4    000007fc     --HOLE--

__llvm_prf_cnts 
*          0    20000000    00000000     UNINITIALIZED

MODULE SUMMARY

       Module                         code    ro data   rw data
       ------                         ----    -------   -------
    .\
       enet_udpecho_client_lwip.obj   1128    0         25     
       startup_ccs.obj                12      512       0      
    +--+------------------------------+-------+---------+---------+
       Total:                         1140    512       25     
                                                               
    .\drivers\
       pinout.obj                     620     0         0      
    +--+------------------------------+-------+---------+---------+
       Total:                         620     0         0      
                                                               
    .\utils\
       lwiplib.obj                    36014   72        97006  
       ustdlib.obj                    1218    22        0      
       uartstdio.obj                  1032    46        5      
    +--+------------------------------+-------+---------+---------+
       Total:                         38264   140       97011  
                                                               
    C:/ti/TivaWare_C_Series-2.2.0.295/driverlib/ccs/Debug/driverlib.lib
       sysctl.obj                     770     596       0      
       emac.obj                       692     24        0      
       gpio.obj                       468     0         0      
       interrupt.obj                  156     176       0      
       systick.obj                    56      0         0      
       flash.obj                      20      0         0      
       cpu.obj                        12      0         0      
    +--+------------------------------+-------+---------+---------+
       Total:                         2174    796       0      
                                                               
    C:\ti\ccs1011\ccs\tools\compiler\ti-cgt-arm_20.2.4.LTS\lib\rtsv7M4_T_le_v4SPD16_eabi.lib
       memcpy_t2.asm.obj              156     0         0      
       memset_t2.asm.obj              122     0         0      
       copy_decompress_lzss.c.obj     104     0         0      
       autoinit.c.obj                 68      0         0      
       u_divt2.asm.obj                64      0         0      
       boot_cortex_m.c.obj            52      0         0      
       memcmp.c.obj                   36      0         0      
       strlen.c.obj                   20      0         0      
       copy_decompress_none.c.obj     14      0         0      
       copy_zero_init.c.obj           12      0         0      
       exit.c.obj                     4       0         0      
       pre_init.c.obj                 4       0         0      
       div0.asm.obj                   2       0         0      
    +--+------------------------------+-------+---------+---------+
       Total:                         658     0         0      
                                                               
       Stack:                         0       0         2048   
       Linker Generated:              0       83        0      
    +--+------------------------------+-------+---------+---------+
       Grand Total:                   42856   1531      99084  


LINKER GENERATED COPY TABLES

__TI_cinit_table @ 0000ad70 records: 2, size/record: 8, table size: 16
	.data: load addr=0000ad28, load size=0000002f bytes, run addr=200182a0, run size=00000070 bytes, compression=lzss
	.bss: load addr=0000ad68, load size=00000008 bytes, run addr=20000000, run size=00017a9f bytes, compression=zero_init


LINKER GENERATED HANDLER TABLE

__TI_handler_table @ 0000ad58 records: 3, size/record: 4, table size: 12
	index: 0, handler: __TI_decompress_lzss
	index: 1, handler: __TI_decompress_none
	index: 2, handler: __TI_zero_init


GLOBAL SYMBOLS: SORTED ALPHABETICALLY BY Name 

address   name                          
-------   ----                          
0000a973  C$$EXIT                       
0000a8f9  CPUcpsie                      
000098cd  DisplayIPAddress              
0000a5d1  EMACAddrGet                   
0000a049  EMACConfigGet                 
00009ec1  EMACConfigSet                 
0000a88d  EMACFrameFilterSet            
00008d29  EMACInit                      
0000a07d  EMACIntClear                  
00009e11  EMACIntEnable                 
0000a1d1  EMACIntStatus                 
000093e1  EMACPHYConfigSet              
0000a325  EMACPHYRead                   
0000a34b  EMACPHYWrite                  
0000a935  EMACPowerManagementStatusGet  
0000a765  EMACReset                     
0000a945  EMACRxDMADescriptorListSet    
0000a77b  EMACRxEnable                  
0000a94b  EMACTimestampIntStatus        
0000a951  EMACTxDMADescriptorListSet    
0000a93d  EMACTxDMAPollDemand           
0000a791  EMACTxEnable                  
0000a815  FlashUserGet                  
0000a1fd  GPIODirModeSet                
00005401  GPIOPadConfigSet              
0000a957  GPIOPinRead                   
0000a7a7  GPIOPinTypeEthernetLED        
0000a6d1  GPIOPinTypeGPIOOutput         
0000a95d  GPIOPinWrite                  
00004a9d  InitDMADescriptors            
000090b9  IntEnable                     
0000a89d  IntMasterEnable               
0000a371  IntPrioritySet                
0000307d  PinoutSet                     
0000a963  ResetISR                      
00003da5  SysCtlClockFreqSet            
0000a969  SysCtlDelay                   
0000a905  SysCtlMOSCConfigSet           
00009ef9  SysCtlPeripheralReady         
0000978d  SysCtlPeripheralReset         
0000a829  SysTickEnable                 
0000a83d  SysTickIntEnable              
0000a851  SysTickIntHandler             
0000a8ad  SysTickPeriodSet              
00008e19  UARTStdioConfig               
0000a395  UARTprintf                    
000025c1  UARTvprintf                   
00009259  UARTwrite                     
0000556d  UdpClientInit                 
00009ce5  UdpEchoRecv                   
200182a0  __STACK_END                   
00000800  __STACK_SIZE                  
200182a0  __STACK_TOP                   
0000ad70  __TI_CINIT_Base               
0000ad80  __TI_CINIT_Limit              
0000ad58  __TI_Handler_Table_Base       
0000ad64  __TI_Handler_Table_Limit      
00009acd  __TI_auto_init_nobinit_nopinit
00009121  __TI_decompress_lzss          
0000a8dd  __TI_decompress_none          
ffffffff  __TI_pprof_out_hndl           
ffffffff  __TI_prof_data_size           
ffffffff  __TI_prof_data_start          
00000000  __TI_static_base__            
0000a911  __TI_zero_init                
00008d27  __aeabi_idiv0                 
00008d27  __aeabi_ldiv0                 
00008cad  __aeabi_memclr                
00008cad  __aeabi_memclr4               
00008cad  __aeabi_memclr8               
00008395  __aeabi_memcpy                
00008395  __aeabi_memcpy4               
00008395  __aeabi_memcpy8               
00008caf  __aeabi_memset                
00008caf  __aeabi_memset4               
00008caf  __aeabi_memset8               
00009c65  __aeabi_uidiv                 
00009c65  __aeabi_uidivmod              
ffffffff  __binit__                     
ffffffff  __c_args__                    
UNDEFED   __mpu_init                    
20017aa0  __stack                       
20000000  __start___llvm_prf_cnts       
20000000  __stop___llvm_prf_cnts        
0000a0b1  _c_int00_noargs               
UNDEFED   _system_post_cinit            
0000a96f  _system_pre_init              
0000a973  abort                         
00007bc5  autoip_arp_reply              
0000a4d1  autoip_network_changed        
000084c9  autoip_start                  
0000a7d3  autoip_stop                   
000056c9  autoip_tmr                    
ffffffff  binit                         
20017a4c  current_header                
20017a50  current_iphdr_dest            
20017a54  current_iphdr_src             
20017a58  current_netif                 
0000a117  dhcp_arp_reply                
000097dd  dhcp_coarse_tmr               
00009599  dhcp_fine_tmr                 
00009321  dhcp_network_changed          
00006929  dhcp_release                  
00007901  dhcp_renew                    
20017a38  dhcp_rx_options_given         
200179e0  dhcp_rx_options_val           
0000645d  dhcp_start                    
0000973b  dhcp_stop                     
000092bd  etharp_cleanup_netif          
00004c4d  etharp_output                 
00004561  etharp_query                  
00006151  etharp_raw                    
00009fa1  etharp_request                
000070f9  etharp_tmr                    
0000ad07  ethbroadcast                  
00006655  ethernet_input                
0000ad0d  ethzero                       
200182d8  g_RxDescList                  
200182e8  g_TxDescList                  
20017a9c  g_bLED                        
20017650  g_pRxDescriptors              
200172f0  g_pTxDescriptors              
20017a5c  g_pfnTimerHandler             
00000000  g_pfnVectors                  
20017a44  g_scbFlag                     
20017a60  g_ui32AbnormalInts            
20017a64  g_ui32IPAddress               
200182a4  g_ui32LocalTimer              
20017a68  g_ui32NormalInts              
20017a6c  g_ui32SysClock                
2001830c  g_ui32ipAddrValid             
0000a7e9  icmp_dest_unreach             
000041a1  icmp_input                    
0000a71d  inet_chksum                   
000081b5  inet_chksum_pbuf              
00008f73  ip4_addr_isbroadcast          
0000ad14  ip_addr_any                   
0000ad18  ip_addr_broadcast             
00002b65  ip_input                      
00009919  ip_output                     
0000683d  ip_output_if                  
000088a9  ip_route                      
0000a735  ipaddr_addr                   
00003b9f  ipaddr_aton                   
00008681  lwIPEthernetIntHandler        
0000855d  lwIPHostTimerHandler          
0000674d  lwIPInit                      
0000a645  lwIPLocalIPAddrGet            
0000a2fd  lwIPTimer                     
0000a229  lwip_htonl                    
0000a401  lwip_htons                    
0000a4f1  lwip_init                     
0000a91d  lwip_ntohl                    
0000a8bd  lwip_ntohs                    
20017770  lwip_stats                    
00004385  main                          
00008799  mem_free                      
00008bb5  mem_init                      
00004f91  mem_malloc                    
00004df5  mem_trim                      
0000a425  memcmp                        
00008395  memcpy                        
000095ed  memp_free                     
00006255  memp_init                     
00007f1d  memp_malloc                   
00008cb5  memset                        
000089b1  netif_add                     
20017a70  netif_default                 
0000867f  netif_init                    
20017a74  netif_list                    
0000a2a9  netif_set_addr                
0000a865  netif_set_default             
0000a175  netif_set_down                
0000a661  netif_set_gw                  
000071b9  netif_set_ipaddr              
0000a449  netif_set_link_down           
00009641  netif_set_link_up             
0000a67d  netif_set_netmask             
00009dd5  netif_set_up                  
00003991  pbuf_alloc                    
00009a85  pbuf_cat                      
0000a7ff  pbuf_chain                    
0000a1a3  pbuf_clen                     
00005d01  pbuf_copy                     
00006a11  pbuf_copy_partial             
00007fc5  pbuf_free                     
20017a9d  pbuf_free_ooseq_pending       
00006cc5  pbuf_header                   
0000762d  pbuf_realloc                  
0000a46b  pbuf_ref                      
00007a65  pbuf_take                     
20000000  ram_heap                      
00007799  raw_input                     
00008e17  stats_init                    
0000a879  strlen                        
0000a8cd  sys_arch_protect              
0000a699  sys_arch_unprotect            
0000a929  sys_now                       
00006f55  sys_timeout                   
0000982d  sys_timeouts_init             
000074b5  tcp_abandon                   
0000a8eb  tcp_abort                     
20017a78  tcp_active_pcbs               
20017a9e  tcp_active_pcbs_changed       
00005bd9  tcp_alloc                     
0000acd2  tcp_backoff                   
20017a7c  tcp_bound_pcbs                
0000a531  tcp_close                     
00009b99  tcp_eff_send_mss              
00005119  tcp_enqueue_flags             
00008821  tcp_fasttmr                   
00008fdf  tcp_init                      
000013d1  tcp_input                     
20017a80  tcp_input_pcb                 
00009439  tcp_keepalive                 
20017a84  tcp_listen_pcbs               
0000a6b5  tcp_next_iss                  
000032e9  tcp_output                    
0000904d  tcp_pcb_purge                 
00008255  tcp_pcb_remove                
0000ad00  tcp_persist_backoff           
00007571  tcp_process_refused_data      
00009e85  tcp_recv_null                 
00009a3d  tcp_recved                    
00008c31  tcp_rexmit                    
000085f1  tcp_rexmit_fast               
0000987d  tcp_rexmit_rto                
00008431  tcp_rst                       
0000a2d3  tcp_seg_copy                  
0000a551  tcp_seg_free                  
0000a571  tcp_segs_free                 
000091f1  tcp_send_empty_ack            
00009383  tcp_send_fin                  
00001951  tcp_slowtmr                   
20017a88  tcp_ticks                     
00009fd9  tcp_timer_needed              
20017a8c  tcp_tmp_pcb                   
0000a591  tcp_tmr                       
20017a90  tcp_tw_pcbs                   
00008da1  tcp_update_rcv_ann_wnd        
00006e7d  tcp_zero_window_probe         
00009bdd  tivaif_init                   
00009491  tivaif_interrupt              
000082f5  tivaif_process_phy_interrupt  
00007279  udp_bind                      
0000870d  udp_connect                   
0000a5b1  udp_disconnect                
000090b7  udp_init                      
000028cd  udp_input                     
0000a48d  udp_new                       
20017a94  udp_pcbs                      
0000a6eb  udp_recv                      
000094e9  udp_remove                    
0000a74d  udp_send                      
00009c21  udp_sendto                    
00005e1d  udp_sendto_if                 
20017a98  upcb                          
0000a0e5  usprintf                      
00009541  ustrncpy                      
00001d99  uvsnprintf                    


GLOBAL SYMBOLS: SORTED BY Symbol Address 

address   name                          
-------   ----                          
00000000  __TI_static_base__            
00000000  g_pfnVectors                  
00000800  __STACK_SIZE                  
000013d1  tcp_input                     
00001951  tcp_slowtmr                   
00001d99  uvsnprintf                    
000025c1  UARTvprintf                   
000028cd  udp_input                     
00002b65  ip_input                      
0000307d  PinoutSet                     
000032e9  tcp_output                    
00003991  pbuf_alloc                    
00003b9f  ipaddr_aton                   
00003da5  SysCtlClockFreqSet            
000041a1  icmp_input                    
00004385  main                          
00004561  etharp_query                  
00004a9d  InitDMADescriptors            
00004c4d  etharp_output                 
00004df5  mem_trim                      
00004f91  mem_malloc                    
00005119  tcp_enqueue_flags             
00005401  GPIOPadConfigSet              
0000556d  UdpClientInit                 
000056c9  autoip_tmr                    
00005bd9  tcp_alloc                     
00005d01  pbuf_copy                     
00005e1d  udp_sendto_if                 
00006151  etharp_raw                    
00006255  memp_init                     
0000645d  dhcp_start                    
00006655  ethernet_input                
0000674d  lwIPInit                      
0000683d  ip_output_if                  
00006929  dhcp_release                  
00006a11  pbuf_copy_partial             
00006cc5  pbuf_header                   
00006e7d  tcp_zero_window_probe         
00006f55  sys_timeout                   
000070f9  etharp_tmr                    
000071b9  netif_set_ipaddr              
00007279  udp_bind                      
000074b5  tcp_abandon                   
00007571  tcp_process_refused_data      
0000762d  pbuf_realloc                  
00007799  raw_input                     
00007901  dhcp_renew                    
00007a65  pbuf_take                     
00007bc5  autoip_arp_reply              
00007f1d  memp_malloc                   
00007fc5  pbuf_free                     
000081b5  inet_chksum_pbuf              
00008255  tcp_pcb_remove                
000082f5  tivaif_process_phy_interrupt  
00008395  __aeabi_memcpy                
00008395  __aeabi_memcpy4               
00008395  __aeabi_memcpy8               
00008395  memcpy                        
00008431  tcp_rst                       
000084c9  autoip_start                  
0000855d  lwIPHostTimerHandler          
000085f1  tcp_rexmit_fast               
0000867f  netif_init                    
00008681  lwIPEthernetIntHandler        
0000870d  udp_connect                   
00008799  mem_free                      
00008821  tcp_fasttmr                   
000088a9  ip_route                      
000089b1  netif_add                     
00008bb5  mem_init                      
00008c31  tcp_rexmit                    
00008cad  __aeabi_memclr                
00008cad  __aeabi_memclr4               
00008cad  __aeabi_memclr8               
00008caf  __aeabi_memset                
00008caf  __aeabi_memset4               
00008caf  __aeabi_memset8               
00008cb5  memset                        
00008d27  __aeabi_idiv0                 
00008d27  __aeabi_ldiv0                 
00008d29  EMACInit                      
00008da1  tcp_update_rcv_ann_wnd        
00008e17  stats_init                    
00008e19  UARTStdioConfig               
00008f73  ip4_addr_isbroadcast          
00008fdf  tcp_init                      
0000904d  tcp_pcb_purge                 
000090b7  udp_init                      
000090b9  IntEnable                     
00009121  __TI_decompress_lzss          
000091f1  tcp_send_empty_ack            
00009259  UARTwrite                     
000092bd  etharp_cleanup_netif          
00009321  dhcp_network_changed          
00009383  tcp_send_fin                  
000093e1  EMACPHYConfigSet              
00009439  tcp_keepalive                 
00009491  tivaif_interrupt              
000094e9  udp_remove                    
00009541  ustrncpy                      
00009599  dhcp_fine_tmr                 
000095ed  memp_free                     
00009641  netif_set_link_up             
0000973b  dhcp_stop                     
0000978d  SysCtlPeripheralReset         
000097dd  dhcp_coarse_tmr               
0000982d  sys_timeouts_init             
0000987d  tcp_rexmit_rto                
000098cd  DisplayIPAddress              
00009919  ip_output                     
00009a3d  tcp_recved                    
00009a85  pbuf_cat                      
00009acd  __TI_auto_init_nobinit_nopinit
00009b99  tcp_eff_send_mss              
00009bdd  tivaif_init                   
00009c21  udp_sendto                    
00009c65  __aeabi_uidiv                 
00009c65  __aeabi_uidivmod              
00009ce5  UdpEchoRecv                   
00009dd5  netif_set_up                  
00009e11  EMACIntEnable                 
00009e85  tcp_recv_null                 
00009ec1  EMACConfigSet                 
00009ef9  SysCtlPeripheralReady         
00009fa1  etharp_request                
00009fd9  tcp_timer_needed              
0000a049  EMACConfigGet                 
0000a07d  EMACIntClear                  
0000a0b1  _c_int00_noargs               
0000a0e5  usprintf                      
0000a117  dhcp_arp_reply                
0000a175  netif_set_down                
0000a1a3  pbuf_clen                     
0000a1d1  EMACIntStatus                 
0000a1fd  GPIODirModeSet                
0000a229  lwip_htonl                    
0000a2a9  netif_set_addr                
0000a2d3  tcp_seg_copy                  
0000a2fd  lwIPTimer                     
0000a325  EMACPHYRead                   
0000a34b  EMACPHYWrite                  
0000a371  IntPrioritySet                
0000a395  UARTprintf                    
0000a401  lwip_htons                    
0000a425  memcmp                        
0000a449  netif_set_link_down           
0000a46b  pbuf_ref                      
0000a48d  udp_new                       
0000a4d1  autoip_network_changed        
0000a4f1  lwip_init                     
0000a531  tcp_close                     
0000a551  tcp_seg_free                  
0000a571  tcp_segs_free                 
0000a591  tcp_tmr                       
0000a5b1  udp_disconnect                
0000a5d1  EMACAddrGet                   
0000a645  lwIPLocalIPAddrGet            
0000a661  netif_set_gw                  
0000a67d  netif_set_netmask             
0000a699  sys_arch_unprotect            
0000a6b5  tcp_next_iss                  
0000a6d1  GPIOPinTypeGPIOOutput         
0000a6eb  udp_recv                      
0000a71d  inet_chksum                   
0000a735  ipaddr_addr                   
0000a74d  udp_send                      
0000a765  EMACReset                     
0000a77b  EMACRxEnable                  
0000a791  EMACTxEnable                  
0000a7a7  GPIOPinTypeEthernetLED        
0000a7d3  autoip_stop                   
0000a7e9  icmp_dest_unreach             
0000a7ff  pbuf_chain                    
0000a815  FlashUserGet                  
0000a829  SysTickEnable                 
0000a83d  SysTickIntEnable              
0000a851  SysTickIntHandler             
0000a865  netif_set_default             
0000a879  strlen                        
0000a88d  EMACFrameFilterSet            
0000a89d  IntMasterEnable               
0000a8ad  SysTickPeriodSet              
0000a8bd  lwip_ntohs                    
0000a8cd  sys_arch_protect              
0000a8dd  __TI_decompress_none          
0000a8eb  tcp_abort                     
0000a8f9  CPUcpsie                      
0000a905  SysCtlMOSCConfigSet           
0000a911  __TI_zero_init                
0000a91d  lwip_ntohl                    
0000a929  sys_now                       
0000a935  EMACPowerManagementStatusGet  
0000a93d  EMACTxDMAPollDemand           
0000a945  EMACRxDMADescriptorListSet    
0000a94b  EMACTimestampIntStatus        
0000a951  EMACTxDMADescriptorListSet    
0000a957  GPIOPinRead                   
0000a95d  GPIOPinWrite                  
0000a963  ResetISR                      
0000a969  SysCtlDelay                   
0000a96f  _system_pre_init              
0000a973  C$$EXIT                       
0000a973  abort                         
0000acd2  tcp_backoff                   
0000ad00  tcp_persist_backoff           
0000ad07  ethbroadcast                  
0000ad0d  ethzero                       
0000ad14  ip_addr_any                   
0000ad18  ip_addr_broadcast             
0000ad58  __TI_Handler_Table_Base       
0000ad64  __TI_Handler_Table_Limit      
0000ad70  __TI_CINIT_Base               
0000ad80  __TI_CINIT_Limit              
20000000  __start___llvm_prf_cnts       
20000000  __stop___llvm_prf_cnts        
20000000  ram_heap                      
200172f0  g_pTxDescriptors              
20017650  g_pRxDescriptors              
20017770  lwip_stats                    
200179e0  dhcp_rx_options_val           
20017a38  dhcp_rx_options_given         
20017a44  g_scbFlag                     
20017a4c  current_header                
20017a50  current_iphdr_dest            
20017a54  current_iphdr_src             
20017a58  current_netif                 
20017a5c  g_pfnTimerHandler             
20017a60  g_ui32AbnormalInts            
20017a64  g_ui32IPAddress               
20017a68  g_ui32NormalInts              
20017a6c  g_ui32SysClock                
20017a70  netif_default                 
20017a74  netif_list                    
20017a78  tcp_active_pcbs               
20017a7c  tcp_bound_pcbs                
20017a80  tcp_input_pcb                 
20017a84  tcp_listen_pcbs               
20017a88  tcp_ticks                     
20017a8c  tcp_tmp_pcb                   
20017a90  tcp_tw_pcbs                   
20017a94  udp_pcbs                      
20017a98  upcb                          
20017a9c  g_bLED                        
20017a9d  pbuf_free_ooseq_pending       
20017a9e  tcp_active_pcbs_changed       
20017aa0  __stack                       
200182a0  __STACK_END                   
200182a0  __STACK_TOP                   
200182a4  g_ui32LocalTimer              
200182d8  g_RxDescList                  
200182e8  g_TxDescList                  
2001830c  g_ui32ipAddrValid             
ffffffff  __TI_pprof_out_hndl           
ffffffff  __TI_prof_data_size           
ffffffff  __TI_prof_data_start          
ffffffff  __binit__                     
ffffffff  __c_args__                    
ffffffff  binit                         
UNDEFED   __mpu_init                    
UNDEFED   _system_post_cinit            

[260 symbols]
